 jaccesswalker-32

 Timestamp is ffffffff (Sun Feb  7 06:28:15 2106)

 Preferred load address is 00400000

 Start         Length     Name                   Class
 0001:00000000 00007000H .text$mn                CODE
 0001:00007000 0000003dH .text$x                 CODE
 0002:00000000 000001b8H .idata$5                DATA
 0002:000001b8 00000004H .00cfg                  DATA
 0002:000001bc 00000004H .CRT$XCA                DATA
 0002:000001c0 00000004H .CRT$XCAA               DATA
 0002:000001c4 00000004H .CRT$XCZ                DATA
 0002:000001c8 00000004H .CRT$XIA                DATA
 0002:000001cc 00000004H .CRT$XIAA               DATA
 0002:000001d0 00000004H .CRT$XIAC               DATA
 0002:000001d4 00000004H .CRT$XIZ                DATA
 0002:000001d8 00000004H .CRT$XPA                DATA
 0002:000001dc 00000004H .CRT$XPZ                DATA
 0002:000001e0 00000004H .CRT$XTA                DATA
 0002:000001e4 0000000cH .CRT$XTZ                DATA
 0002:000001e8 00000000H .gfids$y                DATA
 0002:000001f0 000019f0H .rdata                  DATA
 0002:00001be0 00000130H .rdata$r                DATA
 0002:00001d10 00000008H .rdata$sxdata           DATA
 0002:00001d18 000002f0H .rdata$zzzdbg           DATA
 0002:00002008 00000004H .rtc$IAA                DATA
 0002:0000200c 00000004H .rtc$IZZ                DATA
 0002:00002010 00000004H .rtc$TAA                DATA
 0002:00002014 00000004H .rtc$TZZ                DATA
 0002:00002018 000000fcH .xdata$x                DATA
 0002:00002114 00000000H .edata                  DATA
 0002:00002114 00000104H .idata$2                DATA
 0002:00002218 00000014H .idata$3                DATA
 0002:0000222c 000001b8H .idata$4                DATA
 0002:000023e4 000007feH .idata$6                DATA
 0003:00000000 00000ae8H .data                   DATA
 0003:00000ae8 00000078H .data$r                 DATA
 0003:00000b60 00000690H .bss                    DATA
 0004:00000000 000001d0H .rsrc$01                DATA
 0004:000001d0 00000548H .rsrc$02                DATA

  Address         Publics by Value              Rva+Base       Lib:Object

 0000:00000000       ___guard_longjmp_count     00000000     <absolute>
 0000:00000000       ___guard_fids_count        00000000     <absolute>
 0000:00000000       ___guard_fids_table        00000000     <absolute>
 0000:00000000       ___hybrid_auxiliary_iat    00000000     <absolute>
 0000:00000000       ___guard_iat_count         00000000     <absolute>
 0000:00000000       ___dynamic_value_reloc_table 00000000     <absolute>
 0000:00000000       ___hybrid_code_map         00000000     <absolute>
 0000:00000000       ___enclave_config          00000000     <absolute>
 0000:00000000       ___volatile_metadata       00000000     <absolute>
 0000:00000000       ___guard_iat_table         00000000     <absolute>
 0000:00000000       ___hybrid_code_map_count   00000000     <absolute>
 0000:00000000       ___guard_longjmp_table     00000000     <absolute>
 0000:00000002       ___safe_se_handler_count   00000002     <absolute>
 0000:00000100       ___guard_flags             00000100     <absolute>
 0000:00000000       ___ImageBase               00400000     <linker-defined>
 0001:00000000       _initializeAccessBridge    00401000 f   AccessBridgeCalls.obj
 0001:00000ec0       _shutdownAccessBridge      00401ec0 f   AccessBridgeCalls.obj
 0001:00000f10       _IsJavaWindow              00401f10 f   AccessBridgeCalls.obj
 0001:00000f40       _GetAccessibleContextFromHWND 00401f40 f   AccessBridgeCalls.obj
 0001:00000f70       _getHWNDFromAccessibleContext 00401f70 f   AccessBridgeCalls.obj
 0001:00000fa0       _SetJavaShutdown           00401fa0 f   AccessBridgeCalls.obj
 0001:00000fc0       _SetFocusGained            00401fc0 f   AccessBridgeCalls.obj
 0001:00000fe0       _SetFocusLost              00401fe0 f   AccessBridgeCalls.obj
 0001:00001000       _SetCaretUpdate            00402000 f   AccessBridgeCalls.obj
 0001:00001020       _SetMouseClicked           00402020 f   AccessBridgeCalls.obj
 0001:00001040       _SetMouseEntered           00402040 f   AccessBridgeCalls.obj
 0001:00001060       _SetMouseExited            00402060 f   AccessBridgeCalls.obj
 0001:00001080       _SetMousePressed           00402080 f   AccessBridgeCalls.obj
 0001:000010a0       _SetMouseReleased          004020a0 f   AccessBridgeCalls.obj
 0001:000010c0       _SetMenuCanceled           004020c0 f   AccessBridgeCalls.obj
 0001:000010e0       _SetMenuDeselected         004020e0 f   AccessBridgeCalls.obj
 0001:00001100       _SetMenuSelected           00402100 f   AccessBridgeCalls.obj
 0001:00001120       _SetPopupMenuCanceled      00402120 f   AccessBridgeCalls.obj
 0001:00001140       _SetPopupMenuWillBecomeInvisible 00402140 f   AccessBridgeCalls.obj
 0001:00001160       _SetPopupMenuWillBecomeVisible 00402160 f   AccessBridgeCalls.obj
 0001:00001180       _SetPropertyNameChange     00402180 f   AccessBridgeCalls.obj
 0001:000011a0       _SetPropertyDescriptionChange 004021a0 f   AccessBridgeCalls.obj
 0001:000011c0       _SetPropertyStateChange    004021c0 f   AccessBridgeCalls.obj
 0001:000011e0       _SetPropertyValueChange    004021e0 f   AccessBridgeCalls.obj
 0001:00001200       _SetPropertySelectionChange 00402200 f   AccessBridgeCalls.obj
 0001:00001220       _SetPropertyTextChange     00402220 f   AccessBridgeCalls.obj
 0001:00001240       _SetPropertyCaretChange    00402240 f   AccessBridgeCalls.obj
 0001:00001260       _SetPropertyVisibleDataChange 00402260 f   AccessBridgeCalls.obj
 0001:00001280       _SetPropertyChildChange    00402280 f   AccessBridgeCalls.obj
 0001:000012a0       _SetPropertyActiveDescendentChange 004022a0 f   AccessBridgeCalls.obj
 0001:000012c0       _SetPropertyTableModelChange 004022c0 f   AccessBridgeCalls.obj
 0001:000012e0       _ReleaseJavaObject         004022e0 f   AccessBridgeCalls.obj
 0001:00001310       _GetVersionInfo            00402310 f   AccessBridgeCalls.obj
 0001:00001340       _GetAccessibleContextAt    00402340 f   AccessBridgeCalls.obj
 0001:00001380       _GetAccessibleContextWithFocus 00402380 f   AccessBridgeCalls.obj
 0001:000013b0       _GetAccessibleContextInfo  004023b0 f   AccessBridgeCalls.obj
 0001:000013e0       _GetAccessibleChildFromContext 004023e0 f   AccessBridgeCalls.obj
 0001:00001410       _GetAccessibleParentFromContext 00402410 f   AccessBridgeCalls.obj
 0001:00001440       _GetAccessibleTextInfo     00402440 f   AccessBridgeCalls.obj
 0001:00001480       _GetAccessibleTextItems    00402480 f   AccessBridgeCalls.obj
 0001:000014b0       _GetAccessibleTextSelectionInfo 004024b0 f   AccessBridgeCalls.obj
 0001:000014e0       _GetAccessibleTextAttributes 004024e0 f   AccessBridgeCalls.obj
 0001:00001510       _GetAccessibleTextRect     00402510 f   AccessBridgeCalls.obj
 0001:00001540       _GetAccessibleTextLineBounds 00402540 f   AccessBridgeCalls.obj
 0001:00001580       _GetAccessibleTextRange    00402580 f   AccessBridgeCalls.obj
 0001:000015c0       _getAccessibleTableInfo    004025c0 f   AccessBridgeCalls.obj
 0001:000015f0       _getAccessibleTableCellInfo 004025f0 f   AccessBridgeCalls.obj
 0001:00001630       _getAccessibleTableRowHeader 00402630 f   AccessBridgeCalls.obj
 0001:00001660       _getAccessibleTableColumnHeader 00402660 f   AccessBridgeCalls.obj
 0001:00001690       _getAccessibleTableRowDescription 00402690 f   AccessBridgeCalls.obj
 0001:000016c0       _getAccessibleTableColumnDescription 004026c0 f   AccessBridgeCalls.obj
 0001:000016f0       _getAccessibleTableRowSelectionCount 004026f0 f   AccessBridgeCalls.obj
 0001:00001720       _isAccessibleTableRowSelected 00402720 f   AccessBridgeCalls.obj
 0001:00001750       _getAccessibleTableRowSelections 00402750 f   AccessBridgeCalls.obj
 0001:00001780       _getAccessibleTableColumnSelectionCount 00402780 f   AccessBridgeCalls.obj
 0001:000017b0       _isAccessibleTableColumnSelected 004027b0 f   AccessBridgeCalls.obj
 0001:000017e0       _getAccessibleTableColumnSelections 004027e0 f   AccessBridgeCalls.obj
 0001:00001810       _getAccessibleTableRow     00402810 f   AccessBridgeCalls.obj
 0001:00001840       _getAccessibleTableColumn  00402840 f   AccessBridgeCalls.obj
 0001:00001870       _getAccessibleTableIndex   00402870 f   AccessBridgeCalls.obj
 0001:000018a0       _getAccessibleRelationSet  004028a0 f   AccessBridgeCalls.obj
 0001:000018d0       _getAccessibleHypertext    004028d0 f   AccessBridgeCalls.obj
 0001:00001900       _activateAccessibleHyperlink 00402900 f   AccessBridgeCalls.obj
 0001:00001930       _getAccessibleHyperlinkCount 00402930 f   AccessBridgeCalls.obj
 0001:00001960       _getAccessibleHypertextExt 00402960 f   AccessBridgeCalls.obj
 0001:00001990       _getAccessibleHypertextLinkIndex 00402990 f   AccessBridgeCalls.obj
 0001:000019c0       _getAccessibleHyperlink    004029c0 f   AccessBridgeCalls.obj
 0001:000019f0       _getAccessibleKeyBindings  004029f0 f   AccessBridgeCalls.obj
 0001:00001a20       _getAccessibleIcons        00402a20 f   AccessBridgeCalls.obj
 0001:00001a50       _getAccessibleActions      00402a50 f   AccessBridgeCalls.obj
 0001:00001a80       _doAccessibleActions       00402a80 f   AccessBridgeCalls.obj
 0001:00001ab0       _IsSameObject              00402ab0 f   AccessBridgeCalls.obj
 0001:00001ae0       _setTextContents           00402ae0 f   AccessBridgeCalls.obj
 0001:00001b10       _getParentWithRole         00402b10 f   AccessBridgeCalls.obj
 0001:00001b40       _getParentWithRoleElseRoot 00402b40 f   AccessBridgeCalls.obj
 0001:00001b70       _getTopLevelObject         00402b70 f   AccessBridgeCalls.obj
 0001:00001ba0       _getObjectDepth            00402ba0 f   AccessBridgeCalls.obj
 0001:00001bd0       _getActiveDescendent       00402bd0 f   AccessBridgeCalls.obj
 0001:00001c00       _GetCurrentAccessibleValueFromContext 00402c00 f   AccessBridgeCalls.obj
 0001:00001c30       _GetMaximumAccessibleValueFromContext 00402c30 f   AccessBridgeCalls.obj
 0001:00001c60       _GetMinimumAccessibleValueFromContext 00402c60 f   AccessBridgeCalls.obj
 0001:00001c90       _GetAccessibleSelectionFromContext 00402c90 f   AccessBridgeCalls.obj
 0001:00001cc0       _GetAccessibleSelectionCountFromContext 00402cc0 f   AccessBridgeCalls.obj
 0001:00001cf0       _IsAccessibleChildSelectedFromContext 00402cf0 f   AccessBridgeCalls.obj
 0001:00001d20       _RemoveAccessibleSelectionFromContext 00402d20 f   AccessBridgeCalls.obj
 0001:00001d50       _SelectAllAccessibleSelectionFromContext 00402d50 f   AccessBridgeCalls.obj
 0001:00001d80       _getVirtualAccessibleName  00402d80 f   AccessBridgeCalls.obj
 0001:00001db0       _requestFocus              00402db0 f   AccessBridgeCalls.obj
 0001:00001de0       _selectTextRange           00402de0 f   AccessBridgeCalls.obj
 0001:00001e10       _getTextAttributesInRange  00402e10 f   AccessBridgeCalls.obj
 0001:00001e50       _getVisibleChildrenCount   00402e50 f   AccessBridgeCalls.obj
 0001:00001e80       _getVisibleChildren        00402e80 f   AccessBridgeCalls.obj
 0001:00001eb0       _setCaretPosition          00402eb0 f   AccessBridgeCalls.obj
 0001:00001ee0       _getCaretLocation          00402ee0 f   AccessBridgeCalls.obj
 0001:00001f10       _getEventsWaiting          00402f10 f   AccessBridgeCalls.obj
 0001:00001f30       _addAccessibleSelectionFromContext 00402f30 f   AccessBridgeCalls.obj
 0001:00001f60       _clearAccessibleSelectionFromContext 00402f60 f   AccessBridgeCalls.obj
 0001:00001fa0       _printError                00402fa0 f   AccessBridgeDebug.obj
 0001:000020b0       _PrintDebugString          004030b0 f   AccessBridgeDebug.obj
 0001:00002120       _wPrintJavaDebugString     00403120 f   AccessBridgeDebug.obj
 0001:00002190       _wPrintDebugString         00403190 f   AccessBridgeDebug.obj
 0001:00002200       _initializeFileLogger      00403200 f   AccessBridgeDebug.obj
 0001:00002330       _finalizeFileLogger        00403330 f   AccessBridgeDebug.obj
 0001:00002360       _getTimeStamp              00403360 f   AccessBridgeDebug.obj
 0001:000023a0       _PrintJavaDebugString2     004033a0 f   AccessBridgeDebug.obj
 0001:00002410       ___local_stdio_printf_options 00403410 f i AccessBridgeDebug.obj
 0001:00002420       __vfprintf_l               00403420 f i AccessBridgeDebug.obj
 0001:00002450       __vfwprintf_l              00403450 f i AccessBridgeDebug.obj
 0001:00002480       _fprintf                   00403480 f i AccessBridgeDebug.obj
 0001:000024c0       _printf                    004034c0 f i AccessBridgeDebug.obj
 0001:00002500       _vfprintf                  00403500 f i AccessBridgeDebug.obj
 0001:00002520       _vfwprintf                 00403520 f i AccessBridgeDebug.obj
 0001:00002540       ?initBroadcastMessageIDs@@YAHXZ 00403540 f   AccessBridgeMessages.obj
 0001:00002580       ?getTimeAndDate@@YAPADXZ   00403580 f   AccessInfo.obj
 0001:00002630       ?displayAndLog@@YAXPAUHWND__@@HPAU_iobuf@@PADZZ 00403630 f   AccessInfo.obj
 0001:00002710       ?logString@@YAXPAU_iobuf@@PADZZ 00403710 f   AccessInfo.obj
 0001:000027a0       ?getAccessibleInfo@@YAPADJ_JPADH@Z 004037a0 f   AccessInfo.obj
 0001:000027d0       ?getAccessibleInfo@@YAPADJ_JHHPADH@Z 004037d0 f   AccessInfo.obj
 0001:000049d0       ?appendToBuffer@@YAHPADI0ZZ 004059d0 f   AccessInfo.obj
 0001:00004ab0       __vsnprintf_l              00405ab0 f i AccessInfo.obj
 0001:00004b10       __vsprintf_l               00405b10 f i AccessInfo.obj
 0001:00004b30       _sprintf                   00405b30 f i AccessInfo.obj
 0001:00004b70       _vsprintf                  00405b70 f i AccessInfo.obj
 0001:00004b90       _WinMain@16                00405b90 f   jaccesswalker.obj
 0001:00004c20       ??0AccessibleNode@@QAE@J_JPAV0@PAUHWND__@@PAU_TREEITEM@@@Z 00405c20 f   jaccesswalker.obj
 0001:00004c70       ??1AccessibleNode@@QAE@XZ  00405c70 f   jaccesswalker.obj
 0001:00004ca0       ?setAccessibleName@AccessibleNode@@QAEXPAD@Z 00405ca0 f   jaccesswalker.obj
 0001:00004cd0       ?setAccessibleRole@AccessibleNode@@QAEXPAD@Z 00405cd0 f   jaccesswalker.obj
 0001:00004d00       ?displayAPIWindow@AccessibleNode@@QAEHXZ 00405d00 f   jaccesswalker.obj
 0001:00004e30       ??0Jaccesswalker@@QAE@H@Z  00405e30 f   jaccesswalker.obj
 0001:00004ff0       ?buildAccessibilityTree@Jaccesswalker@@QAEXXZ 00405ff0 f   jaccesswalker.obj
 0001:00005020       ?addComponentNodes@Jaccesswalker@@QAEXJ_JPAVAccessibleNode@@PAUHWND__@@PAU_TREEITEM@@2@Z 00406020 f   jaccesswalker.obj
 0001:00005320       ?WinProc@@YGJPAUHWND__@@IIJ@Z 00406320 f   jaccesswalker.obj
 0001:000055f0       ?EnumWndProc@@YGHPAUHWND__@@J@Z 004065f0 f   jaccesswalker.obj
 0001:000056f0       ?EnumChildProc@@YGHPAUHWND__@@J@Z 004066f0 f   jaccesswalker.obj
 0001:00005790       ?CreateATreeView@@YAPAUHWND__@@PAU1@@Z 00406790 f   jaccesswalker.obj
 0001:00005800       ?AccessInfoWindowProc@@YGJPAUHWND__@@IIJ@Z 00406800 f   jaccesswalker.obj
 0001:00005900       ?IsInaccessibleJavaWindow@@YAHQAUHWND__@@@Z 00406900 f   jaccesswalker.obj
 0001:000060a9       ??_U@YAPAXI@Z              004070a9 f   MSVCRT:new_array.obj
 0001:000060b2       ??_V@YAXPAX@Z              004070b2 f   MSVCRT:delete_array.obj
 0001:000060b7       ___raise_securityfailure   004070b7 f   MSVCRT:gs_report.obj
 0001:000060df       ___report_gsfailure        004070df f   MSVCRT:gs_report.obj
 0001:000061d8       ___report_rangecheckfailure 004071d8 f   MSVCRT:gs_report.obj
 0001:000061e4       ___report_securityfailure  004071e4 f   MSVCRT:gs_report.obj
 0001:000062c0       __aulldiv                  004072c0 f   MSVCRT:ulldiv.obj
 0001:00006328       @__security_check_cookie@4 00407328 f   MSVCRT:secchk.obj
 0001:00006340       __chkstk                   00407340 f   MSVCRT:chkstk.obj
 0001:00006340       __alloca_probe             00407340 f   MSVCRT:chkstk.obj
 0001:0000636d       ??2@YAPAXI@Z               0040736d f   MSVCRT:new_scalar.obj
 0001:0000639d       ??3@YAXPAXI@Z              0040739d f   MSVCRT:delete_scalar_size.obj
 0001:000065ec       _WinMainCRTStartup         004075ec f   MSVCRT:exe_winmain.obj
 0001:000065f6       ??3@YAXPAX@Z               004075f6 f   MSVCRT:delete_scalar.obj
 0001:000065fb       ??0bad_alloc@std@@QAE@ABV01@@Z 004075fb f i MSVCRT:throw_bad_alloc.obj
 0001:00006616       ??0bad_alloc@std@@QAE@XZ   00407616 f i MSVCRT:throw_bad_alloc.obj
 0001:0000662e       ??0bad_array_new_length@std@@QAE@ABV01@@Z 0040762e f i MSVCRT:throw_bad_alloc.obj
 0001:00006649       ??0bad_array_new_length@std@@QAE@XZ 00407649 f i MSVCRT:throw_bad_alloc.obj
 0001:00006661       ??0exception@std@@QAE@ABV01@@Z 00407661 f i MSVCRT:throw_bad_alloc.obj
 0001:0000668d       ??1bad_alloc@std@@UAE@XZ   0040768d f i MSVCRT:throw_bad_alloc.obj
 0001:0000668d       ??1bad_array_new_length@std@@UAE@XZ 0040768d f i MSVCRT:throw_bad_alloc.obj
 0001:0000669e       ??_Eexception@std@@UAEPAXI@Z 0040769e f i MSVCRT:throw_bad_alloc.obj
 0001:0000669e       ??_Ebad_alloc@std@@UAEPAXI@Z 0040769e f i MSVCRT:throw_bad_alloc.obj
 0001:0000669e       ??_Gexception@std@@UAEPAXI@Z 0040769e f i MSVCRT:throw_bad_alloc.obj
 0001:0000669e       ??_Gbad_alloc@std@@UAEPAXI@Z 0040769e f i MSVCRT:throw_bad_alloc.obj
 0001:0000669e       ??_Ebad_array_new_length@std@@UAEPAXI@Z 0040769e f i MSVCRT:throw_bad_alloc.obj
 0001:0000669e       ??_Gbad_array_new_length@std@@UAEPAXI@Z 0040769e f i MSVCRT:throw_bad_alloc.obj
 0001:000066cb       ?__scrt_throw_std_bad_alloc@@YAXXZ 004076cb f   MSVCRT:throw_bad_alloc.obj
 0001:000066e8       ?__scrt_throw_std_bad_array_new_length@@YAXXZ 004076e8 f   MSVCRT:throw_bad_alloc.obj
 0001:00006705       ?what@exception@std@@UBEPBDXZ 00407705 f i MSVCRT:throw_bad_alloc.obj
 0001:00006756       ___scrt_acquire_startup_lock 00407756 f   MSVCRT:utility.obj
 0001:00006788       ___scrt_initialize_crt     00407788 f   MSVCRT:utility.obj
 0001:000067c1       ___scrt_initialize_onexit_tables 004077c1 f   MSVCRT:utility.obj
 0001:00006866       ___scrt_is_nonwritable_in_current_image 00407866 f   MSVCRT:utility.obj
 0001:000068fa       ___scrt_release_startup_lock 004078fa f   MSVCRT:utility.obj
 0001:00006917       ___scrt_uninitialize_crt   00407917 f   MSVCRT:utility.obj
 0001:0000693f       __onexit                   0040793f f   MSVCRT:utility.obj
 0001:0000697a       _atexit                    0040797a f   MSVCRT:utility.obj
 0001:000069dc       ___security_init_cookie    004079dc f   MSVCRT:gs_support.obj
 0001:00006a27       __get_startup_commit_mode  00407a27 f   MSVCRT:commit_mode.obj
 0001:00006a27       __get_startup_thread_locale_mode 00407a27 f   MSVCRT:thread_locale.obj
 0001:00006a27       __get_startup_new_mode     00407a27 f   MSVCRT:new_mode.obj
 0001:00006a27       ___scrt_initialize_winrt   00407a27 f   MSVCRT:utility_desktop.obj
 0001:00006a27       __matherr                  00407a27 f   MSVCRT:matherr.obj
 0001:00006a27       ___scrt_stub_for_initialize_mta 00407a27 f   MSVCRT:utility_desktop.obj
 0001:00006a27       ___scrt_exe_initialize_mta 00407a27 f   MSVCRT:utility_desktop.obj
 0001:00006a2a       __get_startup_argv_mode    00407a2a f   MSVCRT:argv_mode.obj
 0001:00006a2e       __get_startup_file_mode    00407a2e f   MSVCRT:file_mode.obj
 0001:00006a34       ?__scrt_initialize_type_info@@YAXXZ 00407a34 f   MSVCRT:tncleanup.obj
 0001:00006a40       __should_initialize_environment 00407a40 f   MSVCRT:env_mode.obj
 0001:00006a40       ___scrt_stub_for_acrt_initialize 00407a40 f   MSVCRT:ucrt_stubs.obj
 0001:00006a40       ___vcrt_uninitialize       00407a40 f   MSVCRT:ucrt_stubs.obj
 0001:00006a40       ___acrt_initialize         00407a40 f   MSVCRT:ucrt_stubs.obj
 0001:00006a40       ___acrt_uninitialize       00407a40 f   MSVCRT:ucrt_stubs.obj
 0001:00006a40       ___scrt_stub_for_acrt_uninitialize 00407a40 f   MSVCRT:ucrt_stubs.obj
 0001:00006a40       ___vcrt_initialize         00407a40 f   MSVCRT:ucrt_stubs.obj
 0001:00006a43       __initialize_default_precision 00407a43 f   MSVCRT:default_precision.obj
 0001:00006a64       __initialize_invalid_parameter_handler 00407a64 f   MSVCRT:invalid_parameter_handler.obj
 0001:00006a64       __initialize_denormal_control 00407a64 f   MSVCRT:denormal_control.obj
 0001:00006a64       @_guard_check_icall_nop@4  00407a64 f   MSVCRT:guard_support.obj
 0001:00006a65       ___local_stdio_scanf_options 00407a65 f i MSVCRT:default_local_stdio_options.obj
 0001:00006a6b       ___scrt_initialize_default_local_stdio_options 00407a6b f   MSVCRT:default_local_stdio_options.obj
 0001:00006a88       ___scrt_is_user_matherr_present 00407a88 f   MSVCRT:matherr_detection.obj
 0001:00006a94       ___scrt_get_dyn_tls_init_callback 00407a94 f   MSVCRT:dyn_tls_init.obj
 0001:00006a9a       ___scrt_get_dyn_tls_dtor_callback 00407a9a f   MSVCRT:dyn_tls_dtor.obj
 0001:00006aa0       ___scrt_fastfail           00407aa0 f   MSVCRT:utility_desktop.obj
 0001:00006bba       ___scrt_get_show_window_mode 00407bba f   MSVCRT:utility_desktop.obj
 0001:00006beb       ___scrt_initialize_mta     00407beb f   MSVCRT:utility_desktop.obj
 0001:00006bf0       ___scrt_is_managed_app     00407bf0 f   MSVCRT:utility_desktop.obj
 0001:00006c33       ___scrt_set_unhandled_exception_filter 00407c33 f   MSVCRT:utility_desktop.obj
 0001:00006c3f       ___scrt_unhandled_exception_filter@4 00407c3f f   MSVCRT:utility_desktop.obj
 0001:00006c80       __crt_debugger_hook        00407c80 f   MSVCRT:utility_desktop.obj
 0001:00006c88       __RTC_Initialize           00407c88 f   MSVCRT:initsect.obj
 0001:00006cb4       __RTC_Terminate            00407cb4 f   MSVCRT:initsect.obj
 0001:00006ce0       __SEH_prolog4              00407ce0 f   MSVCRT:sehprolg4.obj
 0001:00006d26       __SEH_epilog4              00407d26 f   MSVCRT:sehprolg4.obj
 0001:00006d3b       __except_handler4          00407d3b f   MSVCRT:chandler4gs.obj
 0001:00006d5e       ??_Etype_info@@UAEPAXI@Z   00407d5e f i MSVCRT:std_type_info_static.obj
 0001:00006d5e       ??_Gtype_info@@UAEPAXI@Z   00407d5e f i MSVCRT:std_type_info_static.obj
 0001:00006d81       ___isa_available_init      00407d81 f   MSVCRT:cpu_disp.obj
 0001:00006f18       ___scrt_is_ucrt_dll_in_use 00407f18 f   MSVCRT:ucrt_detection.obj
 0001:00006f24       _IsProcessorFeaturePresent@4 00407f24 f   kernel32:KERNEL32.dll
 0001:00006f2a       _memcpy                    00407f2a f   vcruntime:VCRUNTIME140.dll
 0001:00006f30       _memset                    00407f30 f   vcruntime:VCRUNTIME140.dll
 0001:00006f36       ___CxxFrameHandler3        00407f36 f   vcruntime:VCRUNTIME140.dll
 0001:00006f3c       ___std_exception_copy      00407f3c f   vcruntime:VCRUNTIME140.dll
 0001:00006f42       ___std_exception_destroy   00407f42 f   vcruntime:VCRUNTIME140.dll
 0001:00006f48       __CxxThrowException@8      00407f48 f   vcruntime:VCRUNTIME140.dll
 0001:00006f4e       __except_handler4_common   00407f4e f   vcruntime:VCRUNTIME140.dll
 0001:00006f54       _strlen                    00407f54 f   ucrt:api-ms-win-crt-string-l1-1-0.dll
 0001:00006f5a       _strcpy                    00407f5a f   ucrt:api-ms-win-crt-string-l1-1-0.dll
 0001:00006f60       _strcmp                    00407f60 f   ucrt:api-ms-win-crt-string-l1-1-0.dll
 0001:00006f66       __callnewh                 00407f66 f   ucrt:api-ms-win-crt-heap-l1-1-0.dll
 0001:00006f6c       _malloc                    00407f6c f   ucrt:api-ms-win-crt-heap-l1-1-0.dll
 0001:00006f72       __seh_filter_exe           00407f72 f   ucrt:api-ms-win-crt-runtime-l1-1-0.dll
 0001:00006f78       __set_app_type             00407f78 f   ucrt:api-ms-win-crt-runtime-l1-1-0.dll
 0001:00006f7e       ___setusermatherr          00407f7e f   ucrt:api-ms-win-crt-math-l1-1-0.dll
 0001:00006f84       __configure_narrow_argv    00407f84 f   ucrt:api-ms-win-crt-runtime-l1-1-0.dll
 0001:00006f8a       __initialize_narrow_environment 00407f8a f   ucrt:api-ms-win-crt-runtime-l1-1-0.dll
 0001:00006f90       __get_narrow_winmain_command_line 00407f90 f   ucrt:api-ms-win-crt-runtime-l1-1-0.dll
 0001:00006f96       __initterm                 00407f96 f   ucrt:api-ms-win-crt-runtime-l1-1-0.dll
 0001:00006f9c       __initterm_e               00407f9c f   ucrt:api-ms-win-crt-runtime-l1-1-0.dll
 0001:00006fa2       _exit                      00407fa2 f   ucrt:api-ms-win-crt-runtime-l1-1-0.dll
 0001:00006fa8       __exit                     00407fa8 f   ucrt:api-ms-win-crt-runtime-l1-1-0.dll
 0001:00006fae       __set_fmode                00407fae f   ucrt:api-ms-win-crt-stdio-l1-1-0.dll
 0001:00006fb4       __cexit                    00407fb4 f   ucrt:api-ms-win-crt-runtime-l1-1-0.dll
 0001:00006fba       __c_exit                   00407fba f   ucrt:api-ms-win-crt-runtime-l1-1-0.dll
 0001:00006fc0       __register_thread_local_exe_atexit_callback 00407fc0 f   ucrt:api-ms-win-crt-runtime-l1-1-0.dll
 0001:00006fc6       __configthreadlocale       00407fc6 f   ucrt:api-ms-win-crt-locale-l1-1-0.dll
 0001:00006fcc       __set_new_mode             00407fcc f   ucrt:api-ms-win-crt-heap-l1-1-0.dll
 0001:00006fd2       ___p__commode              00407fd2 f   ucrt:api-ms-win-crt-stdio-l1-1-0.dll
 0001:00006fd8       _free                      00407fd8 f   ucrt:api-ms-win-crt-heap-l1-1-0.dll
 0001:00006fde       __initialize_onexit_table  00407fde f   ucrt:api-ms-win-crt-runtime-l1-1-0.dll
 0001:00006fe4       __register_onexit_function 00407fe4 f   ucrt:api-ms-win-crt-runtime-l1-1-0.dll
 0001:00006fea       __crt_atexit               00407fea f   ucrt:api-ms-win-crt-runtime-l1-1-0.dll
 0001:00006ff0       __controlfp_s              00407ff0 f   ucrt:api-ms-win-crt-runtime-l1-1-0.dll
 0001:00006ff6       _terminate                 00407ff6 f   ucrt:api-ms-win-crt-runtime-l1-1-0.dll
 0002:00000000       __imp__InitCommonControlsEx@4 00409000     comctl32:COMCTL32.dll
 0002:00000004       \177COMCTL32_NULL_THUNK_DATA 00409004     comctl32:COMCTL32.dll
 0002:00000008       __imp__GetStockObject@4    00409008     gdi32:GDI32.dll
 0002:0000000c       \177GDI32_NULL_THUNK_DATA  0040900c     gdi32:GDI32.dll
 0002:00000010       __imp__GetModuleHandleW@4  00409010     kernel32:KERNEL32.dll
 0002:00000014       __imp__GetStartupInfoW@4   00409014     kernel32:KERNEL32.dll
 0002:00000018       __imp__IsDebuggerPresent@0 00409018     kernel32:KERNEL32.dll
 0002:0000001c       __imp__InitializeSListHead@4 0040901c     kernel32:KERNEL32.dll
 0002:00000020       __imp__GetCurrentThreadId@0 00409020     kernel32:KERNEL32.dll
 0002:00000024       __imp__GetCurrentProcessId@0 00409024     kernel32:KERNEL32.dll
 0002:00000028       __imp__QueryPerformanceCounter@4 00409028     kernel32:KERNEL32.dll
 0002:0000002c       __imp__IsProcessorFeaturePresent@4 0040902c     kernel32:KERNEL32.dll
 0002:00000030       __imp__TerminateProcess@8  00409030     kernel32:KERNEL32.dll
 0002:00000034       __imp__GetCurrentProcess@0 00409034     kernel32:KERNEL32.dll
 0002:00000038       __imp__SetUnhandledExceptionFilter@4 00409038     kernel32:KERNEL32.dll
 0002:0000003c       __imp__UnhandledExceptionFilter@4 0040903c     kernel32:KERNEL32.dll
 0002:00000040       __imp__FormatMessageA@28   00409040     kernel32:KERNEL32.dll
 0002:00000044       __imp__GetSystemTimeAsFileTime@4 00409044     kernel32:KERNEL32.dll
 0002:00000048       __imp__LoadLibraryA@4      00409048     kernel32:KERNEL32.dll
 0002:0000004c       __imp__GetProcAddress@8    0040904c     kernel32:KERNEL32.dll
 0002:00000050       __imp__FreeLibrary@4       00409050     kernel32:KERNEL32.dll
 0002:00000054       __imp__GetLastError@0      00409054     kernel32:KERNEL32.dll
 0002:00000058       \177KERNEL32_NULL_THUNK_DATA 00409058     kernel32:KERNEL32.dll
 0002:0000005c       __imp__UpdateWindow@4      0040905c     user32:USER32.dll
 0002:00000060       __imp__GetClientRect@8     00409060     user32:USER32.dll
 0002:00000064       __imp__GetCursorPos@4      00409064     user32:USER32.dll
 0002:00000068       __imp__TrackPopupMenu@28   00409068     user32:USER32.dll
 0002:0000006c       __imp__EnumChildWindows@12 0040906c     user32:USER32.dll
 0002:00000070       __imp__EnumWindows@8       00409070     user32:USER32.dll
 0002:00000074       __imp__GetClassNameA@12    00409074     user32:USER32.dll
 0002:00000078       __imp__LoadCursorA@8       00409078     user32:USER32.dll
 0002:0000007c       __imp__LoadIconA@8         0040907c     user32:USER32.dll
 0002:00000080       __imp__RegisterWindowMessageA@4 00409080     user32:USER32.dll
 0002:00000084       __imp__GetSubMenu@8        00409084     user32:USER32.dll
 0002:00000088       __imp__LoadMenuA@8         00409088     user32:USER32.dll
 0002:0000008c       __imp__GetDlgItem@8        0040908c     user32:USER32.dll
 0002:00000090       __imp__EndDialog@8         00409090     user32:USER32.dll
 0002:00000094       __imp__SetWindowPos@28     00409094     user32:USER32.dll
 0002:00000098       __imp__ShowWindow@8        00409098     user32:USER32.dll
 0002:0000009c       __imp__DestroyWindow@4     0040909c     user32:USER32.dll
 0002:000000a0       __imp__CreateWindowExA@48  004090a0     user32:USER32.dll
 0002:000000a4       __imp__RegisterClassExA@4  004090a4     user32:USER32.dll
 0002:000000a8       __imp__PostQuitMessage@4   004090a8     user32:USER32.dll
 0002:000000ac       __imp__DefWindowProcA@16   004090ac     user32:USER32.dll
 0002:000000b0       __imp__SendMessageA@16     004090b0     user32:USER32.dll
 0002:000000b4       __imp__DispatchMessageA@4  004090b4     user32:USER32.dll
 0002:000000b8       __imp__TranslateMessage@4  004090b8     user32:USER32.dll
 0002:000000bc       __imp__GetMessageA@16      004090bc     user32:USER32.dll
 0002:000000c0       __imp__wsprintfA           004090c0     user32:USER32.dll
 0002:000000c4       __imp__SetDlgItemTextA@12  004090c4     user32:USER32.dll
 0002:000000c8       __imp__ScreenToClient@8    004090c8     user32:USER32.dll
 0002:000000cc       \177USER32_NULL_THUNK_DATA 004090cc     user32:USER32.dll
 0002:000000d0       __imp__memcpy              004090d0     vcruntime:VCRUNTIME140.dll
 0002:000000d4       __imp__memset              004090d4     vcruntime:VCRUNTIME140.dll
 0002:000000d8       __imp____CxxFrameHandler3  004090d8     vcruntime:VCRUNTIME140.dll
 0002:000000dc       __imp____std_exception_copy 004090dc     vcruntime:VCRUNTIME140.dll
 0002:000000e0       __imp____std_exception_destroy 004090e0     vcruntime:VCRUNTIME140.dll
 0002:000000e4       __imp___CxxThrowException@8 004090e4     vcruntime:VCRUNTIME140.dll
 0002:000000e8       __imp___except_handler4_common 004090e8     vcruntime:VCRUNTIME140.dll
 0002:000000ec       \177VCRUNTIME140_NULL_THUNK_DATA 004090ec     vcruntime:VCRUNTIME140.dll
 0002:000000f0       __imp__getenv              004090f0     ucrt:api-ms-win-crt-environment-l1-1-0.dll
 0002:000000f4       \177api-ms-win-crt-environment-l1-1-0_NULL_THUNK_DATA 004090f4     ucrt:api-ms-win-crt-environment-l1-1-0.dll
 0002:000000f8       __imp___set_new_mode       004090f8     ucrt:api-ms-win-crt-heap-l1-1-0.dll
 0002:000000fc       __imp__malloc              004090fc     ucrt:api-ms-win-crt-heap-l1-1-0.dll
 0002:00000100       __imp___callnewh           00409100     ucrt:api-ms-win-crt-heap-l1-1-0.dll
 0002:00000104       __imp__free                00409104     ucrt:api-ms-win-crt-heap-l1-1-0.dll
 0002:00000108       \177api-ms-win-crt-heap-l1-1-0_NULL_THUNK_DATA 00409108     ucrt:api-ms-win-crt-heap-l1-1-0.dll
 0002:0000010c       __imp___configthreadlocale 0040910c     ucrt:api-ms-win-crt-locale-l1-1-0.dll
 0002:00000110       \177api-ms-win-crt-locale-l1-1-0_NULL_THUNK_DATA 00409110     ucrt:api-ms-win-crt-locale-l1-1-0.dll
 0002:00000114       __imp____setusermatherr    00409114     ucrt:api-ms-win-crt-math-l1-1-0.dll
 0002:00000118       \177api-ms-win-crt-math-l1-1-0_NULL_THUNK_DATA 00409118     ucrt:api-ms-win-crt-math-l1-1-0.dll
 0002:0000011c       __imp__terminate           0040911c     ucrt:api-ms-win-crt-runtime-l1-1-0.dll
 0002:00000120       __imp___controlfp_s        00409120     ucrt:api-ms-win-crt-runtime-l1-1-0.dll
 0002:00000124       __imp___crt_atexit         00409124     ucrt:api-ms-win-crt-runtime-l1-1-0.dll
 0002:00000128       __imp___register_onexit_function 00409128     ucrt:api-ms-win-crt-runtime-l1-1-0.dll
 0002:0000012c       __imp___initialize_onexit_table 0040912c     ucrt:api-ms-win-crt-runtime-l1-1-0.dll
 0002:00000130       __imp___seh_filter_exe     00409130     ucrt:api-ms-win-crt-runtime-l1-1-0.dll
 0002:00000134       __imp___set_app_type       00409134     ucrt:api-ms-win-crt-runtime-l1-1-0.dll
 0002:00000138       __imp___c_exit             00409138     ucrt:api-ms-win-crt-runtime-l1-1-0.dll
 0002:0000013c       __imp___configure_narrow_argv 0040913c     ucrt:api-ms-win-crt-runtime-l1-1-0.dll
 0002:00000140       __imp___initialize_narrow_environment 00409140     ucrt:api-ms-win-crt-runtime-l1-1-0.dll
 0002:00000144       __imp___get_narrow_winmain_command_line 00409144     ucrt:api-ms-win-crt-runtime-l1-1-0.dll
 0002:00000148       __imp___initterm           00409148     ucrt:api-ms-win-crt-runtime-l1-1-0.dll
 0002:0000014c       __imp___register_thread_local_exe_atexit_callback 0040914c     ucrt:api-ms-win-crt-runtime-l1-1-0.dll
 0002:00000150       __imp__exit                00409150     ucrt:api-ms-win-crt-runtime-l1-1-0.dll
 0002:00000154       __imp___exit               00409154     ucrt:api-ms-win-crt-runtime-l1-1-0.dll
 0002:00000158       __imp___initterm_e         00409158     ucrt:api-ms-win-crt-runtime-l1-1-0.dll
 0002:0000015c       __imp___cexit              0040915c     ucrt:api-ms-win-crt-runtime-l1-1-0.dll
 0002:00000160       \177api-ms-win-crt-runtime-l1-1-0_NULL_THUNK_DATA 00409160     ucrt:api-ms-win-crt-runtime-l1-1-0.dll
 0002:00000164       __imp__fclose              00409164     ucrt:api-ms-win-crt-stdio-l1-1-0.dll
 0002:00000168       __imp____stdio_common_vfwprintf 00409168     ucrt:api-ms-win-crt-stdio-l1-1-0.dll
 0002:0000016c       __imp____acrt_iob_func     0040916c     ucrt:api-ms-win-crt-stdio-l1-1-0.dll
 0002:00000170       __imp____p__commode        00409170     ucrt:api-ms-win-crt-stdio-l1-1-0.dll
 0002:00000174       __imp____stdio_common_vsprintf 00409174     ucrt:api-ms-win-crt-stdio-l1-1-0.dll
 0002:00000178       __imp__fopen               00409178     ucrt:api-ms-win-crt-stdio-l1-1-0.dll
 0002:0000017c       __imp____stdio_common_vfprintf 0040917c     ucrt:api-ms-win-crt-stdio-l1-1-0.dll
 0002:00000180       __imp___set_fmode          00409180     ucrt:api-ms-win-crt-stdio-l1-1-0.dll
 0002:00000184       __imp__fflush              00409184     ucrt:api-ms-win-crt-stdio-l1-1-0.dll
 0002:00000188       \177api-ms-win-crt-stdio-l1-1-0_NULL_THUNK_DATA 00409188     ucrt:api-ms-win-crt-stdio-l1-1-0.dll
 0002:0000018c       __imp__wcscmp              0040918c     ucrt:api-ms-win-crt-string-l1-1-0.dll
 0002:00000190       __imp__strncpy             00409190     ucrt:api-ms-win-crt-string-l1-1-0.dll
 0002:00000194       __imp__strlen              00409194     ucrt:api-ms-win-crt-string-l1-1-0.dll
 0002:00000198       __imp__strcmp              00409198     ucrt:api-ms-win-crt-string-l1-1-0.dll
 0002:0000019c       __imp__strcpy              0040919c     ucrt:api-ms-win-crt-string-l1-1-0.dll
 0002:000001a0       __imp__strncat             004091a0     ucrt:api-ms-win-crt-string-l1-1-0.dll
 0002:000001a4       \177api-ms-win-crt-string-l1-1-0_NULL_THUNK_DATA 004091a4     ucrt:api-ms-win-crt-string-l1-1-0.dll
 0002:000001a8       __imp__asctime             004091a8     ucrt:api-ms-win-crt-time-l1-1-0.dll
 0002:000001ac       __imp___time64             004091ac     ucrt:api-ms-win-crt-time-l1-1-0.dll
 0002:000001b0       __imp___localtime64        004091b0     ucrt:api-ms-win-crt-time-l1-1-0.dll
 0002:000001b4       \177api-ms-win-crt-time-l1-1-0_NULL_THUNK_DATA 004091b4     ucrt:api-ms-win-crt-time-l1-1-0.dll
 0002:000001b8       ___guard_check_icall_fptr  004091b8     MSVCRT:guard_support.obj
 0002:000001bc       ___xc_a                    004091bc     MSVCRT:initializers.obj
 0002:000001c4       ___xc_z                    004091c4     MSVCRT:initializers.obj
 0002:000001c8       ___xi_a                    004091c8     MSVCRT:initializers.obj
 0002:000001d4       ___xi_z                    004091d4     MSVCRT:initializers.obj
 0002:000001d8       ___xp_a                    004091d8     MSVCRT:initializers.obj
 0002:000001dc       ___xp_z                    004091dc     MSVCRT:initializers.obj
 0002:000001e0       ___xt_a                    004091e0     MSVCRT:initializers.obj
 0002:000001e4       ___xt_z                    004091e4     MSVCRT:initializers.obj
 0002:00001a60       ??_7exception@std@@6B@     0040aa60     MSVCRT:throw_bad_alloc.obj
 0002:00001a68       ??_C@_0BC@EOODALEL@Unknown?5exception@ 0040aa68     MSVCRT:throw_bad_alloc.obj
 0002:00001a80       ??_7bad_alloc@std@@6B@     0040aa80     MSVCRT:throw_bad_alloc.obj
 0002:00001a88       ??_C@_0P@GHFPNOJB@bad?5allocation@ 0040aa88     MSVCRT:throw_bad_alloc.obj
 0002:00001a9c       ??_7bad_array_new_length@std@@6B@ 0040aa9c     MSVCRT:throw_bad_alloc.obj
 0002:00001aa4       ??_C@_0BF@KINCDENJ@bad?5array?5new?5length@ 0040aaa4     MSVCRT:throw_bad_alloc.obj
 0002:00001ac0       ??_7type_info@@6B@         0040aac0     MSVCRT:std_type_info_static.obj
 0002:00001b40       __load_config_used         0040ab40     MSVCRT:loadcfg.obj
 0002:00001be0       ??_R4exception@std@@6B@    0040abe0     MSVCRT:throw_bad_alloc.obj
 0002:00001bf4       ??_R3exception@std@@8      0040abf4     MSVCRT:throw_bad_alloc.obj
 0002:00001c04       ??_R2exception@std@@8      0040ac04     MSVCRT:throw_bad_alloc.obj
 0002:00001c0c       ??_R1A@?0A@EA@exception@std@@8 0040ac0c     MSVCRT:throw_bad_alloc.obj
 0002:00001c28       ??_R4bad_alloc@std@@6B@    0040ac28     MSVCRT:throw_bad_alloc.obj
 0002:00001c3c       ??_R3bad_alloc@std@@8      0040ac3c     MSVCRT:throw_bad_alloc.obj
 0002:00001c4c       ??_R2bad_alloc@std@@8      0040ac4c     MSVCRT:throw_bad_alloc.obj
 0002:00001c58       ??_R1A@?0A@EA@bad_alloc@std@@8 0040ac58     MSVCRT:throw_bad_alloc.obj
 0002:00001c74       ??_R4bad_array_new_length@std@@6B@ 0040ac74     MSVCRT:throw_bad_alloc.obj
 0002:00001c88       ??_R3bad_array_new_length@std@@8 0040ac88     MSVCRT:throw_bad_alloc.obj
 0002:00001c98       ??_R2bad_array_new_length@std@@8 0040ac98     MSVCRT:throw_bad_alloc.obj
 0002:00001ca8       ??_R1A@?0A@EA@bad_array_new_length@std@@8 0040aca8     MSVCRT:throw_bad_alloc.obj
 0002:00001cc4       ??_R4type_info@@6B@        0040acc4     MSVCRT:std_type_info_static.obj
 0002:00001cd8       ??_R3type_info@@8          0040acd8     MSVCRT:std_type_info_static.obj
 0002:00001ce8       ??_R2type_info@@8          0040ace8     MSVCRT:std_type_info_static.obj
 0002:00001cf0       ??_R1A@?0A@EA@type_info@@8 0040acf0     MSVCRT:std_type_info_static.obj
 0002:00001d10       ___safe_se_handler_table   0040ad10     <linker-defined>
 0002:00002008       ___rtc_iaa                 0040b008     MSVCRT:initsect.obj
 0002:0000200c       ___rtc_izz                 0040b00c     MSVCRT:initsect.obj
 0002:00002010       ___rtc_taa                 0040b010     MSVCRT:initsect.obj
 0002:00002014       ___rtc_tzz                 0040b014     MSVCRT:initsect.obj
 0002:00002064       __TI2?AVbad_alloc@std@@    0040b064     MSVCRT:throw_bad_alloc.obj
 0002:00002074       __CTA2?AVbad_alloc@std@@   0040b074     MSVCRT:throw_bad_alloc.obj
 0002:00002080       __CT??_R0?AVbad_alloc@std@@@8??0bad_alloc@std@@QAE@ABV01@@Z12 0040b080     MSVCRT:throw_bad_alloc.obj
 0002:0000209c       __CT??_R0?AVexception@std@@@8??0exception@std@@QAE@ABV01@@Z12 0040b09c     MSVCRT:throw_bad_alloc.obj
 0002:000020b8       __TI3?AVbad_array_new_length@std@@ 0040b0b8     MSVCRT:throw_bad_alloc.obj
 0002:000020c8       __CTA3?AVbad_array_new_length@std@@ 0040b0c8     MSVCRT:throw_bad_alloc.obj
 0002:000020d8       __CT??_R0?AVbad_array_new_length@std@@@8??0bad_array_new_length@std@@QAE@ABV01@@Z12 0040b0d8     MSVCRT:throw_bad_alloc.obj
 0002:00002114       __IMPORT_DESCRIPTOR_COMCTL32 0040b114     comctl32:COMCTL32.dll
 0002:00002128       __IMPORT_DESCRIPTOR_GDI32  0040b128     gdi32:GDI32.dll
 0002:0000213c       __IMPORT_DESCRIPTOR_USER32 0040b13c     user32:USER32.dll
 0002:00002150       __IMPORT_DESCRIPTOR_KERNEL32 0040b150     kernel32:KERNEL32.dll
 0002:00002164       __IMPORT_DESCRIPTOR_VCRUNTIME140 0040b164     vcruntime:VCRUNTIME140.dll
 0002:00002178       __IMPORT_DESCRIPTOR_api-ms-win-crt-string-l1-1-0 0040b178     ucrt:api-ms-win-crt-string-l1-1-0.dll
 0002:0000218c       __IMPORT_DESCRIPTOR_api-ms-win-crt-stdio-l1-1-0 0040b18c     ucrt:api-ms-win-crt-stdio-l1-1-0.dll
 0002:000021a0       __IMPORT_DESCRIPTOR_api-ms-win-crt-environment-l1-1-0 0040b1a0     ucrt:api-ms-win-crt-environment-l1-1-0.dll
 0002:000021b4       __IMPORT_DESCRIPTOR_api-ms-win-crt-time-l1-1-0 0040b1b4     ucrt:api-ms-win-crt-time-l1-1-0.dll
 0002:000021c8       __IMPORT_DESCRIPTOR_api-ms-win-crt-heap-l1-1-0 0040b1c8     ucrt:api-ms-win-crt-heap-l1-1-0.dll
 0002:000021dc       __IMPORT_DESCRIPTOR_api-ms-win-crt-runtime-l1-1-0 0040b1dc     ucrt:api-ms-win-crt-runtime-l1-1-0.dll
 0002:000021f0       __IMPORT_DESCRIPTOR_api-ms-win-crt-math-l1-1-0 0040b1f0     ucrt:api-ms-win-crt-math-l1-1-0.dll
 0002:00002204       __IMPORT_DESCRIPTOR_api-ms-win-crt-locale-l1-1-0 0040b204     ucrt:api-ms-win-crt-locale-l1-1-0.dll
 0002:00002218       __NULL_IMPORT_DESCRIPTOR   0040b218     comctl32:COMCTL32.dll
 0003:00000a68       ?depth@@3HA                0040ca68     jaccesswalker.obj
 0003:00000a6c       ?theJaccesswalkerClassName@@3PADA 0040ca6c     jaccesswalker.obj
 0003:00000a80       ?theAccessInfoClassName@@3PADA 0040ca80     jaccesswalker.obj
 0003:00000ac0       ___security_cookie_complement 0040cac0     MSVCRT:gs_cookie.obj
 0003:00000ac4       ___security_cookie         0040cac4     MSVCRT:gs_cookie.obj
 0003:00000ac8       __fltused                  0040cac8     MSVCRT:fltused.obj
 0003:00000acc       ___scrt_native_dllmain_reason 0040cacc     MSVCRT:utility.obj
 0003:00000ad0       ___scrt_default_matherr    0040cad0     MSVCRT:matherr.obj
 0003:00000ae0       ___isa_enabled             0040cae0     MSVCRT:cpu_disp.obj
 0003:00000ae4       ___scrt_ucrt_dll_is_in_use 0040cae4     MSVCRT:ucrt_stubs.obj
 0003:00000ae8       ??_R0?AVbad_alloc@std@@@8  0040cae8     MSVCRT:throw_bad_alloc.obj
 0003:00000b04       ??_R0?AVexception@std@@@8  0040cb04     MSVCRT:throw_bad_alloc.obj
 0003:00000b20       ??_R0?AVbad_array_new_length@std@@@8 0040cb20     MSVCRT:throw_bad_alloc.obj
 0003:00000b48       ??_R0?AVtype_info@@@8      0040cb48     MSVCRT:std_type_info_static.obj
 0003:00000b60       _theAccessBridgeInitializedFlag 0040cb60     AccessBridgeCalls.obj
 0003:00000b68       ?_OptionsStorage@?1??__local_stdio_printf_options@@9@4_KA 0040cb68     AccessBridgeDebug.obj
 0003:00000c78       ?theFromJavaHelloMsgID@@3IA 0040cc78     AccessBridgeMessages.obj
 0003:00000c7c       ?theFromWindowsHelloMsgID@@3IA 0040cc7c     AccessBridgeMessages.obj
 0003:00000c80       ?g_LogStringCallback@@3P6GXPBD@ZA 0040cc80     AccessInfo.obj
 0003:00000cc8       ?ourHwnd@@3PAUHWND__@@A    0040ccc8     jaccesswalker.obj
 0003:00000ccc       ?topLevelWindow@@3PAUHWND__@@A 0040cccc     jaccesswalker.obj
 0003:00000cd0       ?logfile@@3PAU_iobuf@@A    0040ccd0     jaccesswalker.obj
 0003:00000cd4       ?popupMenu@@3PAUHMENU__@@A 0040ccd4     jaccesswalker.obj
 0003:00000cd8       ?theJaccesswalkerWindow@@3PAUHWND__@@A 0040ccd8     jaccesswalker.obj
 0003:00000cdc       ?theTreeControlWindow@@3PAUHWND__@@A 0040ccdc     jaccesswalker.obj
 0003:00000ce0       ?theInstance@@3PAUHINSTANCE__@@A 0040cce0     jaccesswalker.obj
 0003:00000ce4       ?theJaccesswalker@@3PAVJaccesswalker@@A 0040cce4     jaccesswalker.obj
 0003:00000ce8       ?theSelectedNode@@3PAVAccessibleNode@@A 0040cce8     jaccesswalker.obj
 0003:00000cec       ?thePopupNode@@3PAVAccessibleNode@@A 0040ccec     jaccesswalker.obj
 0003:00000cf0       ?theSelectedAccessibleContext@@3_JA 0040ccf0     jaccesswalker.obj
 0003:00000cf8       ?hwndTV@@3PAUHWND__@@A     0040ccf8     jaccesswalker.obj
 0003:0000101c       ___scrt_current_native_startup_state 0040d01c     MSVCRT:utility.obj
 0003:00001020       ___scrt_native_startup_lock 0040d020     MSVCRT:utility.obj
 0003:00001040       ?__type_info_root_node@@3U__type_info_node@@A 0040d040     MSVCRT:tncleanup.obj
 0003:00001048       ?_OptionsStorage@?1??__local_stdio_scanf_options@@9@4_KA 0040d048     MSVCRT:default_local_stdio_options.obj
 0003:00001050       ___scrt_debugger_hook_flag 0040d050     MSVCRT:utility_desktop.obj
 0003:00001054       ___isa_available           0040d054     MSVCRT:cpu_disp.obj
 0003:00001058       ___favor                   0040d058     MSVCRT:cpu_disp.obj
 0003:00001060       _theAccessBridge           0040d060     <common>
 0003:000011e4       _theAccessBridgeInstance   0040d1e4     <common>
 0003:000011e8       ___dyn_tls_dtor_callback   0040d1e8     <common>
 0003:000011ec       ___dyn_tls_init_callback   0040d1ec     <common>

 entry point at        0001:000065ec

 Static symbols

 0000:ffff0000       .debug$S                   00400000     user32:USER32.dll
 0000:ffff0000       .debug$S                   00400000     user32:USER32.dll
 0000:ffff0000       .debug$S                   00400000     user32:USER32.dll
 0000:ffff0000       .debug$S                   00400000     user32:USER32.dll
 0000:ffff0000       .debug$S                   00400000     user32:USER32.dll
 0000:ffff0000       .debug$S                   00400000     user32:USER32.dll
 0000:ffff0000       .debug$S                   00400000     user32:USER32.dll
 0000:ffff0000       .debug$S                   00400000     user32:USER32.dll
 0000:ffff0000       .debug$S                   00400000     user32:USER32.dll
 0000:ffff0000       .debug$S                   00400000     user32:USER32.dll
 0000:ffff0000       .debug$S                   00400000     user32:USER32.dll
 0000:ffff0000       .debug$S                   00400000     user32:USER32.dll
 0000:ffff0000       .debug$S                   00400000     user32:USER32.dll
 0000:ffff0000       .debug$S                   00400000     ucrt:api-ms-win-crt-runtime-l1-1-0.dll
 0000:ffff0000       .debug$S                   00400000     ucrt:api-ms-win-crt-runtime-l1-1-0.dll
 0000:ffff0000       .debug$S                   00400000     ucrt:api-ms-win-crt-runtime-l1-1-0.dll
 0000:ffff0000       .debug$S                   00400000     ucrt:api-ms-win-crt-runtime-l1-1-0.dll
 0000:ffff0000       .debug$S                   00400000     ucrt:api-ms-win-crt-runtime-l1-1-0.dll
 0000:ffff0000       .debug$S                   00400000     ucrt:api-ms-win-crt-runtime-l1-1-0.dll
 0000:ffff0000       .debug$S                   00400000     ucrt:api-ms-win-crt-runtime-l1-1-0.dll
 0000:ffff0000       .debug$S                   00400000     ucrt:api-ms-win-crt-runtime-l1-1-0.dll
 0000:ffff0000       .debug$S                   00400000     ucrt:api-ms-win-crt-heap-l1-1-0.dll
 0000:ffff0000       .debug$S                   00400000     ucrt:api-ms-win-crt-stdio-l1-1-0.dll
 0000:ffff0000       .debug$S                   00400000     ucrt:api-ms-win-crt-heap-l1-1-0.dll
 0000:ffff0000       .debug$S                   00400000     ucrt:api-ms-win-crt-locale-l1-1-0.dll
 0000:ffff0000       .debug$S                   00400000     ucrt:api-ms-win-crt-runtime-l1-1-0.dll
 0000:ffff0000       .debug$S                   00400000     ucrt:api-ms-win-crt-runtime-l1-1-0.dll
 0000:ffff0000       .debug$S                   00400000     ucrt:api-ms-win-crt-runtime-l1-1-0.dll
 0000:ffff0000       .debug$S                   00400000     ucrt:api-ms-win-crt-stdio-l1-1-0.dll
 0000:ffff0000       .debug$S                   00400000     ucrt:api-ms-win-crt-runtime-l1-1-0.dll
 0000:ffff0000       .debug$S                   00400000     ucrt:api-ms-win-crt-runtime-l1-1-0.dll
 0000:ffff0000       .debug$S                   00400000     ucrt:api-ms-win-crt-runtime-l1-1-0.dll
 0000:ffff0000       .debug$S                   00400000     ucrt:api-ms-win-crt-runtime-l1-1-0.dll
 0000:ffff0000       .debug$S                   00400000     ucrt:api-ms-win-crt-runtime-l1-1-0.dll
 0000:ffff0000       .debug$S                   00400000     ucrt:api-ms-win-crt-runtime-l1-1-0.dll
 0000:ffff0000       .debug$S                   00400000     ucrt:api-ms-win-crt-runtime-l1-1-0.dll
 0000:ffff0000       .debug$S                   00400000     ucrt:api-ms-win-crt-math-l1-1-0.dll
 0000:ffff0000       .debug$S                   00400000     ucrt:api-ms-win-crt-runtime-l1-1-0.dll
 0000:ffff0000       .debug$S                   00400000     ucrt:api-ms-win-crt-runtime-l1-1-0.dll
 0000:ffff0000       .debug$S                   00400000     ucrt:api-ms-win-crt-heap-l1-1-0.dll
 0000:ffff0000       .debug$S                   00400000     ucrt:api-ms-win-crt-heap-l1-1-0.dll
 0000:ffff0000       .debug$S                   00400000     ucrt:api-ms-win-crt-string-l1-1-0.dll
 0000:ffff0000       .debug$S                   00400000     ucrt:api-ms-win-crt-string-l1-1-0.dll
 0000:ffff0000       .debug$S                   00400000     ucrt:api-ms-win-crt-time-l1-1-0.dll
 0000:ffff0000       .debug$S                   00400000     ucrt:api-ms-win-crt-time-l1-1-0.dll
 0000:ffff0000       .debug$S                   00400000     ucrt:api-ms-win-crt-time-l1-1-0.dll
 0000:ffff0000       .debug$S                   00400000     ucrt:api-ms-win-crt-stdio-l1-1-0.dll
 0000:ffff0000       .debug$S                   00400000     ucrt:api-ms-win-crt-stdio-l1-1-0.dll
 0000:ffff0000       .debug$S                   00400000     ucrt:api-ms-win-crt-string-l1-1-0.dll
 0000:ffff0000       .debug$S                   00400000     ucrt:api-ms-win-crt-environment-l1-1-0.dll
 0000:ffff0000       .debug$S                   00400000     ucrt:api-ms-win-crt-stdio-l1-1-0.dll
 0000:ffff0000       .debug$S                   00400000     ucrt:api-ms-win-crt-stdio-l1-1-0.dll
 0000:ffff0000       .debug$S                   00400000     ucrt:api-ms-win-crt-stdio-l1-1-0.dll
 0000:ffff0000       .debug$S                   00400000     ucrt:api-ms-win-crt-stdio-l1-1-0.dll
 0000:ffff0000       .debug$S                   00400000     ucrt:api-ms-win-crt-stdio-l1-1-0.dll
 0000:ffff0000       .debug$S                   00400000     ucrt:api-ms-win-crt-string-l1-1-0.dll
 0000:ffff0000       .debug$S                   00400000     ucrt:api-ms-win-crt-string-l1-1-0.dll
 0000:ffff0000       .debug$S                   00400000     ucrt:api-ms-win-crt-string-l1-1-0.dll
 0000:ffff0000       .debug$S                   00400000     user32:USER32.dll
 0000:ffff0000       .debug$S                   00400000     vcruntime:VCRUNTIME140.dll
 0000:ffff0000       .debug$S                   00400000     vcruntime:VCRUNTIME140.dll
 0000:ffff0000       .debug$S                   00400000     vcruntime:VCRUNTIME140.dll
 0000:ffff0000       .debug$S                   00400000     vcruntime:VCRUNTIME140.dll
 0000:ffff0000       .debug$S                   00400000     vcruntime:VCRUNTIME140.dll
 0000:ffff0000       .debug$S                   00400000     vcruntime:VCRUNTIME140.dll
 0000:ffff0000       .debug$S                   00400000     vcruntime:VCRUNTIME140.dll
 0000:ffff0000       .debug$S                   00400000     vcruntime:VCRUNTIME140.dll
 0000:ffff0000       .debug$S                   00400000     user32:USER32.dll
 0000:ffff0000       .debug$S                   00400000     kernel32:KERNEL32.dll
 0000:ffff0000       .debug$S                   00400000     kernel32:KERNEL32.dll
 0000:ffff0000       .debug$S                   00400000     kernel32:KERNEL32.dll
 0000:ffff0000       .debug$S                   00400000     kernel32:KERNEL32.dll
 0000:ffff0000       .debug$S                   00400000     kernel32:KERNEL32.dll
 0000:ffff0000       .debug$S                   00400000     kernel32:KERNEL32.dll
 0000:ffff0000       .debug$S                   00400000     kernel32:KERNEL32.dll
 0000:ffff0000       .debug$S                   00400000     kernel32:KERNEL32.dll
 0000:ffff0000       .debug$S                   00400000     kernel32:KERNEL32.dll
 0000:ffff0000       .debug$S                   00400000     kernel32:KERNEL32.dll
 0000:ffff0000       .debug$S                   00400000     kernel32:KERNEL32.dll
 0000:ffff0000       .debug$S                   00400000     kernel32:KERNEL32.dll
 0000:ffff0000       .debug$S                   00400000     kernel32:KERNEL32.dll
 0000:ffff0000       .debug$S                   00400000     kernel32:KERNEL32.dll
 0000:ffff0000       .debug$S                   00400000     kernel32:KERNEL32.dll
 0000:ffff0000       .debug$S                   00400000     kernel32:KERNEL32.dll
 0000:ffff0000       .debug$S                   00400000     kernel32:KERNEL32.dll
 0000:ffff0000       .debug$S                   00400000     kernel32:KERNEL32.dll
 0000:ffff0000       .debug$S                   00400000     user32:USER32.dll
 0000:ffff0000       .debug$S                   00400000     user32:USER32.dll
 0000:ffff0000       .debug$S                   00400000     user32:USER32.dll
 0000:ffff0000       .debug$S                   00400000     user32:USER32.dll
 0000:ffff0000       .debug$S                   00400000     user32:USER32.dll
 0000:ffff0000       .debug$S                   00400000     user32:USER32.dll
 0000:ffff0000       .debug$S                   00400000     user32:USER32.dll
 0000:ffff0000       .debug$S                   00400000     user32:USER32.dll
 0000:ffff0000       .debug$S                   00400000     comctl32:COMCTL32.dll
 0000:ffff0000       .debug$S                   00400000     user32:USER32.dll
 0000:ffff0000       .debug$S                   00400000     user32:USER32.dll
 0000:ffff0000       .debug$S                   00400000     user32:USER32.dll
 0000:ffff0000       .debug$S                   00400000     user32:USER32.dll
 0000:ffff0000       .debug$S                   00400000     user32:USER32.dll
 0000:ffff0000       .debug$S                   00400000     gdi32:GDI32.dll
 0001:00004990       _localtime                 00405990 f   AccessInfo.obj
 0001:000049b0       _time                      004059b0 f   AccessInfo.obj
 0001:0000556c       $LN26                      0040656c     jaccesswalker.obj
 0001:00005580       $LN25                      00406580     jaccesswalker.obj
 0001:000062c0       $$000000                   004072c0     MSVCRT:ulldiv.obj
 0001:00006340       $$000000                   00407340     MSVCRT:chkstk.obj
 0001:000063ab       ?pre_c_initialization@@YAHXZ 004073ab f   MSVCRT:exe_winmain.obj
 0001:00006456       ?post_pgo_initialization@@YAHXZ 00407456 f   MSVCRT:exe_winmain.obj
 0001:0000645e       ?pre_cpp_initialization@@YAXXZ 0040745e f   MSVCRT:exe_winmain.obj
 0001:00006470       ?__scrt_common_main_seh@@YAHXZ 00407470 f   MSVCRT:exe_winmain.obj
 0001:00006712       ?find_pe_section@@YAPAU_IMAGE_SECTION_HEADER@@QAEI@Z 00407712 f   MSVCRT:utility.obj
 0001:0000698f       ___get_entropy             0040798f f   MSVCRT:gs_support.obj
 0001:00006ce0       $$000000                   00407ce0     MSVCRT:sehprolg4.obj
 0001:00007000       __unwindfunclet$?addComponentNodes@Jaccesswalker@@QAEXJ_JPAVAccessibleNode@@PAUHWND__@@PAU_TREEITEM@@2@Z$0 00408000 f   jaccesswalker.obj
 0001:00007015       __ehhandler$?addComponentNodes@Jaccesswalker@@QAEXJ_JPAVAccessibleNode@@PAUHWND__@@PAU_TREEITEM@@2@Z 00408015 f   jaccesswalker.obj
 0002:000001c0       ?pre_cpp_initializer@@3P6AXXZA 004091c0     MSVCRT:exe_winmain.obj
 0002:000001cc       ?pre_c_initializer@@3P6AHXZA 004091cc     MSVCRT:exe_winmain.obj
 0002:000001d0       ?post_pgo_initializer@@3P6AHXZA 004091d0     MSVCRT:exe_winmain.obj
 0002:000001f0       $SG45876                   004091f0     AccessBridgeDebug.obj
 0002:0000020c       $SG45878                   0040920c     AccessBridgeDebug.obj
 0002:00000214       $SG45879                   00409214     AccessBridgeDebug.obj
 0002:00000218       $SG45881                   00409218     AccessBridgeDebug.obj
 0002:00000220       $SG45882                   00409220     AccessBridgeDebug.obj
 0002:00000238       $SG45909                   00409238     AccessBridgeDebug.obj
 0002:00000254       $SG45910                   00409254     AccessBridgeDebug.obj
 0002:00000260       $SG45912                   00409260     AccessBridgeDebug.obj
 0002:00000264       $SG45954                   00409264     AccessBridgeDebug.obj
 0002:0000026c       $SG45955                   0040926c     AccessBridgeDebug.obj
 0002:00000270       $SG45971                   00409270     AccessBridgeDebug.obj
 0002:00000278       $SG45972                   00409278     AccessBridgeDebug.obj
 0002:0000027c       $SG46014                   0040927c     AccessBridgeDebug.obj
 0002:00000284       $SG46015                   00409284     AccessBridgeDebug.obj
 0002:00000288       $SG46031                   00409288     AccessBridgeDebug.obj
 0002:00000290       $SG46032                   00409290     AccessBridgeDebug.obj
 0002:00000294       $SG40743                   00409294     AccessBridgeMessages.obj
 0002:000002b0       $SG40744                   004092b0     AccessBridgeMessages.obj
 0002:000002d0       $SG50163                   004092d0     AccessInfo.obj
 0002:000002d4       $SG50165                   004092d4     AccessInfo.obj
 0002:000002d8       $SG50168                   004092d8     AccessInfo.obj
 0002:000002e4       $SG50213                   004092e4     AccessInfo.obj
 0002:00000310       $SG50214                   00409310     AccessInfo.obj
 0002:00000314       $SG50215                   00409314     AccessInfo.obj
 0002:00000318       $SG50233                   00409318     AccessInfo.obj
 0002:0000031c       $SG50375                   0040931c     AccessInfo.obj
 0002:00000344       $SG50376                   00409344     AccessInfo.obj
 0002:0000035c       $SG50377                   0040935c     AccessInfo.obj
 0002:00000384       $SG50378                   00409384     AccessInfo.obj
 0002:000003b0       $SG50379                   004093b0     AccessInfo.obj
 0002:000003dc       $SG50380                   004093dc     AccessInfo.obj
 0002:0000040c       $SG50384                   0040940c     AccessInfo.obj
 0002:00000438       $SG50385                   00409438     AccessInfo.obj
 0002:0000045c       $SG50388                   0040945c     AccessInfo.obj
 0002:00000478       $SG50389                   00409478     AccessInfo.obj
 0002:0000047c       $SG50390                   0040947c     AccessInfo.obj
 0002:00000490       $SG50393                   00409490     AccessInfo.obj
 0002:000004b4       $SG50394                   004094b4     AccessInfo.obj
 0002:000004d0       $SG50395                   004094d0     AccessInfo.obj
 0002:000004e8       $SG50396                   004094e8     AccessInfo.obj
 0002:000004fc       $SG50397                   004094fc     AccessInfo.obj
 0002:00000520       $SG50398                   00409520     AccessInfo.obj
 0002:00000534       $SG50399                   00409534     AccessInfo.obj
 0002:00000558       $SG50400                   00409558     AccessInfo.obj
 0002:00000574       $SG50401                   00409574     AccessInfo.obj
 0002:00000590       $SG50402                   00409590     AccessInfo.obj
 0002:000005bc       $SG50405                   004095bc     AccessInfo.obj
 0002:000005e0       $SG50408                   004095e0     AccessInfo.obj
 0002:00000620       $SG50411                   00409620     AccessInfo.obj
 0002:00000644       $SG50412                   00409644     AccessInfo.obj
 0002:00000668       $SG50413                   00409668     AccessInfo.obj
 0002:0000068c       $SG50416                   0040968c     AccessInfo.obj
 0002:0000069c       $SG50419                   0040969c     AccessInfo.obj
 0002:000006d0       $SG50420                   004096d0     AccessInfo.obj
 0002:000006e8       $SG50423                   004096e8     AccessInfo.obj
 0002:0000070c       $SG50424                   0040970c     AccessInfo.obj
 0002:0000072c       $SG50425                   0040972c     AccessInfo.obj
 0002:00000744       $SG50428                   00409744     AccessInfo.obj
 0002:0000076c       $SG50429                   0040976c     AccessInfo.obj
 0002:00000794       $SG50433                   00409794     AccessInfo.obj
 0002:000007b8       $SG50437                   004097b8     AccessInfo.obj
 0002:000007dc       $SG50438                   004097dc     AccessInfo.obj
 0002:000007fc       $SG50439                   004097fc     AccessInfo.obj
 0002:0000081c       $SG50441                   0040981c     AccessInfo.obj
 0002:00000844       $SG50443                   00409844     AccessInfo.obj
 0002:00000860       $SG50446                   00409860     AccessInfo.obj
 0002:000008a4       $SG50449                   004098a4     AccessInfo.obj
 0002:000008e0       $SG50452                   004098e0     AccessInfo.obj
 0002:00000904       $SG50453                   00409904     AccessInfo.obj
 0002:00000924       $SG50454                   00409924     AccessInfo.obj
 0002:00000944       $SG50455                   00409944     AccessInfo.obj
 0002:00000970       $SG50457                   00409970     AccessInfo.obj
 0002:00000990       $SG50458                   00409990     AccessInfo.obj
 0002:000009b4       $SG50459                   004099b4     AccessInfo.obj
 0002:000009d8       $SG50460                   004099d8     AccessInfo.obj
 0002:000009fc       $SG50462                   004099fc     AccessInfo.obj
 0002:00000a18       $SG50463                   00409a18     AccessInfo.obj
 0002:00000a34       $SG50464                   00409a34     AccessInfo.obj
 0002:00000a54       $SG50465                   00409a54     AccessInfo.obj
 0002:00000a70       $SG50466                   00409a70     AccessInfo.obj
 0002:00000a88       $SG50468                   00409a88     AccessInfo.obj
 0002:00000aa4       $SG50469                   00409aa4     AccessInfo.obj
 0002:00000ac4       $SG50470                   00409ac4     AccessInfo.obj
 0002:00000ae0       $SG50473                   00409ae0     AccessInfo.obj
 0002:00000b04       $SG50475                   00409b04     AccessInfo.obj
 0002:00000b2c       $SG50476                   00409b2c     AccessInfo.obj
 0002:00000b4c       $SG50477                   00409b4c     AccessInfo.obj
 0002:00000b68       $SG50478                   00409b68     AccessInfo.obj
 0002:00000b8c       $SG50481                   00409b8c     AccessInfo.obj
 0002:00000bb8       $SG50484                   00409bb8     AccessInfo.obj
 0002:00000bdc       $SG50485                   00409bdc     AccessInfo.obj
 0002:00000bfc       $SG50486                   00409bfc     AccessInfo.obj
 0002:00000c1c       $SG50488                   00409c1c     AccessInfo.obj
 0002:00000c40       $SG50490                   00409c40     AccessInfo.obj
 0002:00000c5c       $SG50492                   00409c5c     AccessInfo.obj
 0002:00000c78       $SG50494                   00409c78     AccessInfo.obj
 0002:00000c94       $SG50498                   00409c94     AccessInfo.obj
 0002:00000cbc       $SG50499                   00409cbc     AccessInfo.obj
 0002:00000cd8       $SG50500                   00409cd8     AccessInfo.obj
 0002:00000cfc       $SG50501                   00409cfc     AccessInfo.obj
 0002:00000d20       $SG50502                   00409d20     AccessInfo.obj
 0002:00000d44       $SG50503                   00409d44     AccessInfo.obj
 0002:00000d60       $SG50504                   00409d60     AccessInfo.obj
 0002:00000d80       $SG50507                   00409d80     AccessInfo.obj
 0002:00000dac       $SG50508                   00409dac     AccessInfo.obj
 0002:00000dd8       $SG50509                   00409dd8     AccessInfo.obj
 0002:00000dec       $SG50510                   00409dec     AccessInfo.obj
 0002:00000e04       $SG50511                   00409e04     AccessInfo.obj
 0002:00000e20       $SG50512                   00409e20     AccessInfo.obj
 0002:00000e38       $SG50515                   00409e38     AccessInfo.obj
 0002:00000e7c       $SG50518                   00409e7c     AccessInfo.obj
 0002:00000ea0       $SG50519                   00409ea0     AccessInfo.obj
 0002:00000eb4       $SG50520                   00409eb4     AccessInfo.obj
 0002:00000ec8       $SG50523                   00409ec8     AccessInfo.obj
 0002:00000ef8       $SG50524                   00409ef8     AccessInfo.obj
 0002:00000f20       $SG50525                   00409f20     AccessInfo.obj
 0002:00000f44       $SG50526                   00409f44     AccessInfo.obj
 0002:00000f6c       $SG50527                   00409f6c     AccessInfo.obj
 0002:00000f8c       $SG50530                   00409f8c     AccessInfo.obj
 0002:00000fc0       $SG50531                   00409fc0     AccessInfo.obj
 0002:00000fd8       $SG50532                   00409fd8     AccessInfo.obj
 0002:00000fdc       $SG50535                   00409fdc     AccessInfo.obj
 0002:00001008       $SG50536                   0040a008     AccessInfo.obj
 0002:0000102c       $SG50537                   0040a02c     AccessInfo.obj
 0002:00001040       $SG50538                   0040a040     AccessInfo.obj
 0002:00001058       $SG50539                   0040a058     AccessInfo.obj
 0002:00001074       $SG50540                   0040a074     AccessInfo.obj
 0002:0000108c       $SG50543                   0040a08c     AccessInfo.obj
 0002:000010b8       $SG50546                   0040a0b8     AccessInfo.obj
 0002:000010dc       $SG50547                   0040a0dc     AccessInfo.obj
 0002:000010f0       $SG50548                   0040a0f0     AccessInfo.obj
 0002:00001104       $SG50550                   0040a104     AccessInfo.obj
 0002:00001128       $SG50552                   0040a128     AccessInfo.obj
 0002:00001150       $SG50553                   0040a150     AccessInfo.obj
 0002:00001170       $SG50554                   0040a170     AccessInfo.obj
 0002:00001188       $SG50556                   0040a188     AccessInfo.obj
 0002:000011ac       $SG50557                   0040a1ac     AccessInfo.obj
 0002:000011cc       $SG50558                   0040a1cc     AccessInfo.obj
 0002:000011e8       $SG50559                   0040a1e8     AccessInfo.obj
 0002:0000120c       $SG50561                   0040a20c     AccessInfo.obj
 0002:00001248       $SG50564                   0040a248     AccessInfo.obj
 0002:00001268       $SG50566                   0040a268     AccessInfo.obj
 0002:00001284       $SG50567                   0040a284     AccessInfo.obj
 0002:0000129c       $SG50568                   0040a29c     AccessInfo.obj
 0002:000012b8       $SG50570                   0040a2b8     AccessInfo.obj
 0002:000012c0       $SG50571                   0040a2c0     AccessInfo.obj
 0002:000012cc       $SG50572                   0040a2cc     AccessInfo.obj
 0002:000012ec       $SG50573                   0040a2ec     AccessInfo.obj
 0002:000012f4       $SG50574                   0040a2f4     AccessInfo.obj
 0002:00001300       $SG50575                   0040a300     AccessInfo.obj
 0002:00001308       $SG50576                   0040a308     AccessInfo.obj
 0002:00001314       $SG50577                   0040a314     AccessInfo.obj
 0002:00001324       $SG50578                   0040a324     AccessInfo.obj
 0002:0000132c       $SG50579                   0040a32c     AccessInfo.obj
 0002:0000133c       $SG50580                   0040a33c     AccessInfo.obj
 0002:00001350       $SG50581                   0040a350     AccessInfo.obj
 0002:00001358       $SG50582                   0040a358     AccessInfo.obj
 0002:00001364       $SG50583                   0040a364     AccessInfo.obj
 0002:00001374       $SG50584                   0040a374     AccessInfo.obj
 0002:0000137c       $SG50585                   0040a37c     AccessInfo.obj
 0002:00001388       $SG50586                   0040a388     AccessInfo.obj
 0002:00001398       $SG50587                   0040a398     AccessInfo.obj
 0002:000013a0       $SG50588                   0040a3a0     AccessInfo.obj
 0002:000013c4       $SG50589                   0040a3c4     AccessInfo.obj
 0002:000013e8       $SG50590                   0040a3e8     AccessInfo.obj
 0002:00001404       $SG50591                   0040a404     AccessInfo.obj
 0002:00001420       $SG50592                   0040a420     AccessInfo.obj
 0002:00001444       $SG50593                   0040a444     AccessInfo.obj
 0002:00001460       $SG50594                   0040a460     AccessInfo.obj
 0002:0000147c       $SG50595                   0040a47c     AccessInfo.obj
 0002:00001498       $SG50596                   0040a498     AccessInfo.obj
 0002:000014b4       $SG50597                   0040a4b4     AccessInfo.obj
 0002:000014d0       $SG50598                   0040a4d0     AccessInfo.obj
 0002:000014f8       $SG50601                   0040a4f8     AccessInfo.obj
 0002:00001518       $SG50602                   0040a518     AccessInfo.obj
 0002:00001544       $SG50603                   0040a544     AccessInfo.obj
 0002:00001560       $SG50605                   0040a560     AccessInfo.obj
 0002:00001598       $SG50607                   0040a598     AccessInfo.obj
 0002:000015d4       $SG50610                   0040a5d4     AccessInfo.obj
 0002:000015f4       $SG50612                   0040a5f4     AccessInfo.obj
 0002:00001610       $SG50613                   0040a610     AccessInfo.obj
 0002:00001628       $SG50614                   0040a628     AccessInfo.obj
 0002:00001644       $SG50616                   0040a644     AccessInfo.obj
 0002:0000164c       $SG50617                   0040a64c     AccessInfo.obj
 0002:00001658       $SG50618                   0040a658     AccessInfo.obj
 0002:00001678       $SG50619                   0040a678     AccessInfo.obj
 0002:00001680       $SG50620                   0040a680     AccessInfo.obj
 0002:0000168c       $SG50621                   0040a68c     AccessInfo.obj
 0002:00001694       $SG50622                   0040a694     AccessInfo.obj
 0002:000016a0       $SG50623                   0040a6a0     AccessInfo.obj
 0002:000016b0       $SG50624                   0040a6b0     AccessInfo.obj
 0002:000016b8       $SG50625                   0040a6b8     AccessInfo.obj
 0002:000016c8       $SG50626                   0040a6c8     AccessInfo.obj
 0002:000016dc       $SG50627                   0040a6dc     AccessInfo.obj
 0002:000016e4       $SG50628                   0040a6e4     AccessInfo.obj
 0002:000016f0       $SG50629                   0040a6f0     AccessInfo.obj
 0002:00001700       $SG50630                   0040a700     AccessInfo.obj
 0002:00001708       $SG50631                   0040a708     AccessInfo.obj
 0002:00001714       $SG50632                   0040a714     AccessInfo.obj
 0002:00001724       $SG50633                   0040a724     AccessInfo.obj
 0002:0000172c       $SG50634                   0040a72c     AccessInfo.obj
 0002:00001750       $SG50635                   0040a750     AccessInfo.obj
 0002:00001774       $SG50636                   0040a774     AccessInfo.obj
 0002:00001790       $SG50637                   0040a790     AccessInfo.obj
 0002:000017ac       $SG50638                   0040a7ac     AccessInfo.obj
 0002:000017d0       $SG50639                   0040a7d0     AccessInfo.obj
 0002:000017ec       $SG50640                   0040a7ec     AccessInfo.obj
 0002:00001808       $SG50641                   0040a808     AccessInfo.obj
 0002:00001824       $SG50642                   0040a824     AccessInfo.obj
 0002:00001840       $SG50643                   0040a840     AccessInfo.obj
 0002:0000185c       $SG50644                   0040a85c     AccessInfo.obj
 0002:00001884       $SG50647                   0040a884     AccessInfo.obj
 0002:000018a4       $SG50648                   0040a8a4     AccessInfo.obj
 0002:000018d0       $SG58027                   0040a8d0     jaccesswalker.obj
 0002:000018d2       $SG58075                   0040a8d2     jaccesswalker.obj
 0002:000018d3       $SG58149                   0040a8d3     jaccesswalker.obj
 0002:000018d4       $SG58028                   0040a8d4     jaccesswalker.obj
 0002:000018e6       $SG58252                   0040a8e6     jaccesswalker.obj
 0002:000018e8       $SG58029                   0040a8e8     jaccesswalker.obj
 0002:00001908       $SG58115                   0040a908     jaccesswalker.obj
 0002:00001914       $SG58150                   0040a914     jaccesswalker.obj
 0002:0000191c       $SG58178                   0040a91c     jaccesswalker.obj
 0002:00001924       $SG58179                   0040a924     jaccesswalker.obj
 0002:0000193c       $SG58202                   0040a93c     jaccesswalker.obj
 0002:00001948       $SG58209                   0040a948     jaccesswalker.obj
 0002:00001954       $SG58213                   0040a954     jaccesswalker.obj
 0002:00001960       $SG58215                   0040a960     jaccesswalker.obj
 0002:0000196c       $SG58218                   0040a96c     jaccesswalker.obj
 0002:00001978       $SG58220                   0040a978     jaccesswalker.obj
 0002:00001988       $SG58222                   0040a988     jaccesswalker.obj
 0002:00001994       $SG58227                   0040a994     jaccesswalker.obj
 0002:000019a0       $SG58229                   0040a9a0     jaccesswalker.obj
 0002:000019ac       $SG58232                   0040a9ac     jaccesswalker.obj
 0002:000019b8       $SG58253                   0040a9b8     jaccesswalker.obj
 0002:000019c8       $SG58299                   0040a9c8     jaccesswalker.obj
 0002:000019cc       $SG58300                   0040a9cc     jaccesswalker.obj
 0002:000019d0       $SG58301                   0040a9d0     jaccesswalker.obj
 0002:000019dc       $SG58332                   0040a9dc     jaccesswalker.obj
 0002:000019f8       $SG58302                   0040a9f8     jaccesswalker.obj
 0002:00001a38       $SG58334                   0040aa38     jaccesswalker.obj
 0002:00001a54       _GS_ExceptionPointers      0040aa54     MSVCRT:gs_report.obj
 0002:00002018       __unwindtable$?addComponentNodes@Jaccesswalker@@QAEXJ_JPAVAccessibleNode@@PAUHWND__@@PAU_TREEITEM@@2@Z 0040b018     jaccesswalker.obj
 0002:00002020       __ehfuncinfo$?addComponentNodes@Jaccesswalker@@QAEXJ_JPAVAccessibleNode@@PAUHWND__@@PAU_TREEITEM@@2@Z 0040b020     jaccesswalker.obj
 0002:00002048       __sehtable$?__scrt_common_main_seh@@YAHXZ 0040b048     MSVCRT:exe_winmain.obj
 0002:000020f8       __sehtable$___scrt_is_nonwritable_in_current_image 0040b0f8     MSVCRT:utility.obj
 0002:000023fc       .idata$6                   0040b3fc     comctl32:COMCTL32.dll
 0002:0000241c       .idata$6                   0040b41c     gdi32:GDI32.dll
 0002:000025f0       .idata$6                   0040b5f0     user32:USER32.dll
 0002:0000277c       .idata$6                   0040b77c     kernel32:KERNEL32.dll
 0002:00002816       .idata$6                   0040b816     vcruntime:VCRUNTIME140.dll
 0002:00002ad6       .idata$6                   0040bad6     ucrt:api-ms-win-crt-string-l1-1-0.dll
 0002:00002af8       .idata$6                   0040baf8     ucrt:api-ms-win-crt-stdio-l1-1-0.dll
 0002:00002b18       .idata$6                   0040bb18     ucrt:api-ms-win-crt-environment-l1-1-0.dll
 0002:00002b3e       .idata$6                   0040bb3e     ucrt:api-ms-win-crt-time-l1-1-0.dll
 0002:00002b5e       .idata$6                   0040bb5e     ucrt:api-ms-win-crt-heap-l1-1-0.dll
 0002:00002b7e       .idata$6                   0040bb7e     ucrt:api-ms-win-crt-runtime-l1-1-0.dll
 0002:00002ba0       .idata$6                   0040bba0     ucrt:api-ms-win-crt-math-l1-1-0.dll
 0002:00002bc0       .idata$6                   0040bbc0     ucrt:api-ms-win-crt-locale-l1-1-0.dll
 0003:00000000       $SG46583                   0040c000     AccessBridgeCalls.obj
 0003:00000018       $SG46587                   0040c018     AccessBridgeCalls.obj
 0003:00000024       $SG46589                   0040c024     AccessBridgeCalls.obj
 0003:00000038       $SG46591                   0040c038     AccessBridgeCalls.obj
 0003:0000004c       $SG46593                   0040c04c     AccessBridgeCalls.obj
 0003:0000005c       $SG46595                   0040c05c     AccessBridgeCalls.obj
 0003:00000070       $SG46597                   0040c070     AccessBridgeCalls.obj
 0003:00000084       $SG46599                   0040c084     AccessBridgeCalls.obj
 0003:00000098       $SG46601                   0040c098     AccessBridgeCalls.obj
 0003:000000ac       $SG46603                   0040c0ac     AccessBridgeCalls.obj
 0003:000000c0       $SG46605                   0040c0c0     AccessBridgeCalls.obj
 0003:000000d4       $SG46607                   0040c0d4     AccessBridgeCalls.obj
 0003:000000e8       $SG46609                   0040c0e8     AccessBridgeCalls.obj
 0003:000000fc       $SG46611                   0040c0fc     AccessBridgeCalls.obj
 0003:00000110       $SG46613                   0040c110     AccessBridgeCalls.obj
 0003:00000128       $SG46615                   0040c128     AccessBridgeCalls.obj
 0003:0000014c       $SG46617                   0040c14c     AccessBridgeCalls.obj
 0003:0000016c       $SG46619                   0040c16c     AccessBridgeCalls.obj
 0003:00000184       $SG46621                   0040c184     AccessBridgeCalls.obj
 0003:000001a4       $SG46623                   0040c1a4     AccessBridgeCalls.obj
 0003:000001c0       $SG46625                   0040c1c0     AccessBridgeCalls.obj
 0003:000001dc       $SG46627                   0040c1dc     AccessBridgeCalls.obj
 0003:000001fc       $SG46629                   0040c1fc     AccessBridgeCalls.obj
 0003:00000214       $SG46631                   0040c214     AccessBridgeCalls.obj
 0003:00000230       $SG46633                   0040c230     AccessBridgeCalls.obj
 0003:00000250       $SG46635                   0040c250     AccessBridgeCalls.obj
 0003:0000026c       $SG46637                   0040c26c     AccessBridgeCalls.obj
 0003:00000290       $SG46639                   0040c290     AccessBridgeCalls.obj
 0003:000002b0       $SG46641                   0040c2b0     AccessBridgeCalls.obj
 0003:000002c4       $SG46643                   0040c2c4     AccessBridgeCalls.obj
 0003:000002d4       $SG46645                   0040c2d4     AccessBridgeCalls.obj
 0003:000002e4       $SG46647                   0040c2e4     AccessBridgeCalls.obj
 0003:000002f4       $SG46649                   0040c2f4     AccessBridgeCalls.obj
 0003:00000314       $SG46651                   0040c314     AccessBridgeCalls.obj
 0003:00000334       $SG46653                   0040c334     AccessBridgeCalls.obj
 0003:0000034c       $SG46655                   0040c34c     AccessBridgeCalls.obj
 0003:0000036c       $SG46657                   0040c36c     AccessBridgeCalls.obj
 0003:00000388       $SG46659                   0040c388     AccessBridgeCalls.obj
 0003:000003a8       $SG46661                   0040c3a8     AccessBridgeCalls.obj
 0003:000003c8       $SG46663                   0040c3c8     AccessBridgeCalls.obj
 0003:000003e0       $SG46665                   0040c3e0     AccessBridgeCalls.obj
 0003:000003fc       $SG46667                   0040c3fc     AccessBridgeCalls.obj
 0003:00000418       $SG46669                   0040c418     AccessBridgeCalls.obj
 0003:00000438       $SG46671                   0040c438     AccessBridgeCalls.obj
 0003:0000045c       $SG46673                   0040c45c     AccessBridgeCalls.obj
 0003:00000480       $SG46675                   0040c480     AccessBridgeCalls.obj
 0003:000004a4       $SG46677                   0040c4a4     AccessBridgeCalls.obj
 0003:000004c4       $SG46679                   0040c4c4     AccessBridgeCalls.obj
 0003:000004e4       $SG46681                   0040c4e4     AccessBridgeCalls.obj
 0003:0000050c       $SG46683                   0040c50c     AccessBridgeCalls.obj
 0003:0000052c       $SG46685                   0040c52c     AccessBridgeCalls.obj
 0003:00000550       $SG46687                   0040c550     AccessBridgeCalls.obj
 0003:00000568       $SG46689                   0040c568     AccessBridgeCalls.obj
 0003:00000584       $SG46691                   0040c584     AccessBridgeCalls.obj
 0003:0000059c       $SG46693                   0040c59c     AccessBridgeCalls.obj
 0003:000005b8       $SG46695                   0040c5b8     AccessBridgeCalls.obj
 0003:000005d0       $SG46697                   0040c5d0     AccessBridgeCalls.obj
 0003:000005ec       $SG46699                   0040c5ec     AccessBridgeCalls.obj
 0003:00000608       $SG46701                   0040c608     AccessBridgeCalls.obj
 0003:00000624       $SG46703                   0040c624     AccessBridgeCalls.obj
 0003:00000644       $SG46705                   0040c644     AccessBridgeCalls.obj
 0003:0000065c       $SG46707                   0040c65c     AccessBridgeCalls.obj
 0003:00000678       $SG46709                   0040c678     AccessBridgeCalls.obj
 0003:0000068c       $SG46711                   0040c68c     AccessBridgeCalls.obj
 0003:000006a4       $SG46713                   0040c6a4     AccessBridgeCalls.obj
 0003:000006b8       $SG46715                   0040c6b8     AccessBridgeCalls.obj
 0003:000006d0       $SG46717                   0040c6d0     AccessBridgeCalls.obj
 0003:000006e8       $SG46719                   0040c6e8     AccessBridgeCalls.obj
 0003:00000708       $SG46721                   0040c708     AccessBridgeCalls.obj
 0003:00000724       $SG46723                   0040c724     AccessBridgeCalls.obj
 0003:0000073c       $SG46725                   0040c73c     AccessBridgeCalls.obj
 0003:00000758       $SG46727                   0040c758     AccessBridgeCalls.obj
 0003:00000770       $SG46729                   0040c770     AccessBridgeCalls.obj
 0003:00000798       $SG46731                   0040c798     AccessBridgeCalls.obj
 0003:000007c0       $SG46733                   0040c7c0     AccessBridgeCalls.obj
 0003:000007e8       $SG46735                   0040c7e8     AccessBridgeCalls.obj
 0003:0000080c       $SG46737                   0040c80c     AccessBridgeCalls.obj
 0003:00000830       $SG46739                   0040c830     AccessBridgeCalls.obj
 0003:00000854       $SG46741                   0040c854     AccessBridgeCalls.obj
 0003:0000087c       $SG46743                   0040c87c     AccessBridgeCalls.obj
 0003:000008a4       $SG46745                   0040c8a4     AccessBridgeCalls.obj
 0003:000008cc       $SG46747                   0040c8cc     AccessBridgeCalls.obj
 0003:000008f4       $SG46749                   0040c8f4     AccessBridgeCalls.obj
 0003:00000904       $SG46751                   0040c904     AccessBridgeCalls.obj
 0003:00000918       $SG46753                   0040c918     AccessBridgeCalls.obj
 0003:0000092c       $SG46755                   0040c92c     AccessBridgeCalls.obj
 0003:00000948       $SG46757                   0040c948     AccessBridgeCalls.obj
 0003:00000958       $SG46759                   0040c958     AccessBridgeCalls.obj
 0003:0000096c       $SG46761                   0040c96c     AccessBridgeCalls.obj
 0003:00000988       $SG46763                   0040c988     AccessBridgeCalls.obj
 0003:00000998       $SG46765                   0040c998     AccessBridgeCalls.obj
 0003:000009a8       $SG46767                   0040c9a8     AccessBridgeCalls.obj
 0003:000009c4       $SG46769                   0040c9c4     AccessBridgeCalls.obj
 0003:000009dc       $SG46771                   0040c9dc     AccessBridgeCalls.obj
 0003:000009f0       $SG46773                   0040c9f0     AccessBridgeCalls.obj
 0003:00000a04       $SG46775                   0040ca04     AccessBridgeCalls.obj
 0003:00000a18       $SG46777                   0040ca18     AccessBridgeCalls.obj
 0003:00000a2c       ?warning@?1??appendToBuffer@@YAHPADI0ZZ@4PADA 0040ca2c     AccessInfo.obj
 0003:00000a90       ?szAppName@?1???0Jaccesswalker@@QAE@H@Z@4PADA 0040ca90     jaccesswalker.obj
 0003:00000aa0       ?szMenuName@?1???0Jaccesswalker@@QAE@H@Z@4PADA 0040caa0     jaccesswalker.obj
 0003:00000b70       _logFP                     0040cb70     AccessBridgeDebug.obj
 0003:00000b78       ?retbuf@?1??printError@@9@4PADA 0040cb78     AccessBridgeDebug.obj
 0003:00000c88       ?datebuf@?1??getTimeAndDate@@YAPADXZ@4PADA 0040cc88     AccessInfo.obj
 0003:00000d00       _GS_ExceptionRecord        0040cd00     MSVCRT:gs_report.obj
 0003:00000d50       _GS_ContextRecord          0040cd50     MSVCRT:gs_report.obj
 0003:00001024       ?is_initialized_as_dll@@3_NA 0040d024     MSVCRT:utility.obj
 0003:00001025       ?module_local_atexit_table_initialized@@3_NA 0040d025     MSVCRT:utility.obj
 0003:00001028       ?module_local_atexit_table@@3U_onexit_table_t@@A 0040d028     MSVCRT:utility.obj
 0003:00001034       ?module_local_at_quick_exit_table@@3U_onexit_table_t@@A 0040d034     MSVCRT:utility.obj
 0004:000001d0       $R000000                   0040e1d0     jaccesswalker-32.exe.res
 0004:00000260       $R000090                   0040e260     jaccesswalker-32.exe.res
 0004:000002f0       $R000120                   0040e2f0     jaccesswalker-32.exe.res
 0004:00000390       $R0001C0                   0040e390     jaccesswalker-32.exe.res
 0004:000003e0       $R000210                   0040e3e0     jaccesswalker-32.exe.res
